:020000040800F2
:1000000000500020A501000808B54FF00050002165
:10001000014B984708BD00BF0105000873B54FF4B8
:10002000007301AD194C0326ADF80430294618239E
:1000300017488DF806608DF80730A0474FF0200371
:1000400029461448ADF80430A0474FF48063ADF85A
:100050000430294604230E488DF80730A0474FF09E
:10006000400329460B48ADF80430A0478DF80660E0
:1000700029460D3606488DF80760ADF80460A047A4
:1000800003483146044B98477CBD00BF7503000808
:1000900000080140001401400904000808B5084B9D
:1000A0009847012144F22500064B984701214FF45F
:1000B0000030054B984701200146044B984708BD86
:1000C000D9010008C9040008E5040008AD040008CF
:1000D00008B5164B9847164B9847164B9847164944
:1000E0004FF4E1330B604FF000038B80CB800B812A
:1000F0008B814FF00C034B811048114B98470F48F0
:100100000121104B98470CE00F490C48C95C0133A2
:1001100013700E4B9847094880210D4B98470028D3
:10012000F9D00C4A1378232BEED9FEE79D00000886
:10013000090000081D0000082801002000380140C7
:10014000FD020008CD02000814050008E7020008BF
:10015000EF020008200100200C4B0D4A9A420FD0FC
:10016000002303E00A49595899500433074A0949C2
:1001700098188842F6D303E0002243F8042B00E0ED
:10018000054B064A9342F7D3704700BF000000209A
:100190003C0500082001002020010020380100203B
:1001A000FEE70000684620F007018D4601B50023F8
:1001B00082B001E0019B01330193019A034B9A4203
:1001C000F8D9034B9847034B9847FEE71FA1070058
:1001D00059010008D1000008394B82B01A6842F07A
:1001E00001021A605968374A01EA02025A601A6825
:1001F00022F0847222F480321A601A6822F480227B
:100200001A605A6822F4FE025A604FF41F029A6084
:100210000022019200921A6842F480321A60284B40
:100220001B6803F400330093019B01330193009B8F
:100230001BB9019BB3F5A06FF1D1214B1B6813F4DF
:10024000003318BF01230093009B012B35D11E4BB7
:100250001A6842F010021A601A6822F003021A604B
:100260001A6842F002021A60154B5A685A605A68BE
:100270005A605A6842F480625A605A6822F47C12CA
:100280005A605A6842F4E8125A601A6842F0807262
:100290001A600B4B1A6812F0007FFAD05A6822F0ED
:1002A00003025A605A6842F002025A60044B5B68CB
:1002B00003F00C03082BF9D100E0FEE702B0704711
:1002C000001002400000FFF80020024021B18389A5
:1002D0009BB243F4005304E0838923F400531B04CE
:1002E0001B0C83817047C905C90D81807047038845
:1002F00019420CBF0020012070470000038ACA8801
:1003000023F440531B041B0C1343038230B50D46EA
:1003100083890989AA8823F4B05341EA02026989D2
:1003200023F00C030A431B041B0C92B242EA0303A2
:100330008381838AAA8923F440731B041B0C134313
:1003400087B004468382094B01A89847084B2A6866
:100350009C420CBF049B039B5B00B3FBF2F3013395
:100360005B089BB2238107B030BD00BF0D040008BD
:1003700000380140CB78F0B513F0100F18BF8A7821
:10038000098803F00F0C18BF4CEA020C11F0FF0FA4
:100390001AD0046800220126964006EA0105B542FB
:1003A0000ED196000F27B7400CFA06F624EA070490
:1003B0003443282B01D1456102E0482B08BF056179
:1003C0000132082AE7D10460FF291CD944680022C1
:1003D00002F108050126AE4006EA0105B5420ED13C
:1003E00096000F27B7400CFA06F624EA07043443B8
:1003F000282B01D1456102E0482B08BF056101327D
:10040000082AE5D14460F0BD01617047224B10B568
:100410005A6802F00C02042A14D0082A12D15A6831
:10042000596802F47012920C023211F4803F03D02A
:100430005B6813F4003F01D0184B00E0184B5A439F
:10044000026001E0164B0360134B16495A680468BA
:1004500002F0F00212098A5C34FA02F242605C682F
:1004600004F4E06C4FEA1C2C11F80C4032FA04F44E
:1004700084605C6804F4605C4FEADC2C11F80C10BA
:10048000CA40C2605B68084903F440439B0BCB5CE5
:10049000B2FBF3F2026110BD0010024000093D0002
:1004A00000127A00100100200C01002019B1054B48
:1004B0005A69104303E0034B5A6922EA000058616D
:1004C000704700BF0010024019B1054B9A691043F4
:1004D00003E0034B9A6922EA00009861704700BF6D
:1004E0000010024019B1054BDA69104303E0034BD9
:1004F000DA6922EA0000D861704700BF00100240AC
:1005000021F0604121F07F01014B01439960704768
:1005100000ED00E00D0A48656C6C6F20434D5349B7
:10052000532D2D2D2D2D0D0A56312E302E302031EC
:0C053000312F323030390D0A000000007D
:10053C0000500020A5010008000000000000000091
:10054C00A1010008A1010008A101000800000000A1
:10055C00000000000000000000000000A1010008E5
:10056C00A101000800000000A1010008A101000881
:10057C00A1010008A1010008A1010008A1010008C7
:10058C00A1010008A1010008A1010008A1010008B7
:10059C00A1010008A1010008A1010008A1010008A7
:1005AC00A1010008A1010008A1010008A101000897
:1005BC00A1010008A1010008A1010008A101000887
:1005CC00A1010008A1010008A1010008A101000877
:1005DC00A1010008A1010008A1010008A101000867
:1005EC00A1010008A1010008A1010008A101000857
:1005FC00A1010008A1010008A1010008A101000847
:10060C00A1010008A1010008A1010008A101000836
:10061C00A1010008A1010008A101000800000000D0
:10062C0000000000000000000000000000000000BE
:10063C0000000000000000005FF808F1020406084A
:10064C00000000000102030401020304060708096C
:04000005080001A549
:00000001FF
